:100000000C9499010C94241C0C94B6010C94B60128
:100010000C94B6010C94B6010C94B6010C94B60184
:100020000C94B6010C94B6010C9443230C94152443
:100030000C942E1E0C94B6010C94B6010C94B601CF
:100040000C94B6010C94B6010C94B6010C94B60154
:100050000C94B6010C94D21E0C94B6010C94B6010B
:100060000C94B6010C94B6010C94B6010C94B60134
:100070000C94B6010C94B6010C94B6010C94B60124
:100080000C94B6010C94B6010C94B6010C94B60114
:100090000C94B6010C94B6010C94B6010C94B60104
:1000A0000C94B6010C94B6010C94B6016B046B046D
:1000B00097049704FE041C05330633062705C00584
:1000C000D105D1058224A924A125A924A125F5249F
:1000D0001825A1256F257E2535001E001F00200054
:1000E000210022002B0014001A0008001500170040
:1000F000396104001600070009000A00E1001D0034
:100100001B0006001900050029612D002E002F009C
:10011000300000002A002961E200E3004C00015891
:10012000230024002500260027004A001C00180098
:100130000C001200130031000B000D000E000F0028
:100140003341340011001000360037003800E5005C
:1001500000005000510052004F004D00E4004B00E1
:100160004E00E60028002C00005C0000AC00AE0051
:10017000AB0000000100A900B600ED00B700F900D7
:100180000100AA00EF00EE00F000FA0000003A00C3
:100190003B003C003D00000001003E003F004000ED
:1001A00041000000F100F200010001000100010027
:1001B000BD002400250026000000005CBE002100D8
:1001C000220023000000420057001E001F002000F4
:1001D0005600430055002700000001005400440071
:1001E00000000100010001000100450001004A007B
:1001F0004D002A6401000100160344004100430041
:10020000540059004C005F005200410048000000BB
:100210001403720061006C007000680069006500E2
:100220003000320000000403090409023B0002010F
:1002300000A0FA09040000010301010009211101D5
:1002400000012240000705810308000109040100A4
:100250000103000000092111010001227B000705B4
:1002600082032000011201000200000008EDFE6080
:100270003001000102000105010902A10185020906
:1002800001A1000509190129081500250195087526
:100290000181020501093009311581257F9502751B
:1002A00008810609381581257F95017508810605A5
:1002B0000C0A38021581257F950175088106C0C09A
:1002C00005010980A101850319012AB7001501263E
:1002D000B700950175108100C0050C0901A10185C9
:1002E0000419012AA002150126A0029501751081AA
:1002F00000C005010906A101050719E029E715005D
:100300002501950875018102950175088101050790
:10031000190029FF150026FF0095067508810005C4
:10032000081901290595057501910295017503913B
:1003300001C011241FBECFEFDAE0DEBFCDBF11E058
:10034000A0E0B1E0EEEDFCE402C005900D92A03A11
:10035000B107D9F722E0A0EAB1E001C01D92AD3BA0
:10036000B207E1F70E9422150C946D260C94000050
:1003700081E0089581E008950C94BA0108950C94E9
:10038000BE011F93CF93DF9300D000D01F92CDB753
:10039000DEB749835A836B833091A30189819A81A7
:1003A000311114C0662359F0222349F00E947208CB
:1003B000182F682F89819A810E94190803C00E9412
:1003C0004508182F69817A81812F04C00E94720824
:1003D00069817A810F900F900F900F900F90DF91AD
:1003E000CF911F910C94C50FFC01262F40815181A4
:1003F0006281738184810C94C10181E00895CF935F
:10040000DF93EC0160E00E94F401BE01DF91CF9127
:100410000C94BF010C9432110C942E1108950E947B
:10042000C3060E940E022FEF84E39CE0215080401F
:100430009040E1F700C000000C94F81E0F931F934A
:10044000CF93DF938C0161E00E94F401EC01B801CD
:100450000E94BC018823F1F1B801CE010E94311B3A
:100460008823C1F1B801CE010E94D017882391F1F1
:10047000B801CE010E948D1A882361F1F8018281B2
:10048000882309F1CB358DE5D807C1F050F4C115AB
:10049000FCE5DF0781F0CF3DDC45A9F40E94D30DD8
:1004A00019C0CC35EDE5DE0761F0CD35DD4559F4F9
:1004B0000E941C0D08C00E940F020CC00E94250D56
:1004C00002C00E94280DC801DF91CF911F910F91AA
:1004D0000C94B80180E0DF91CF911F910F910895A6
:1004E0000E94111E0C9489020E948C020C94171E0B
:1004F00008950C94780281E008950C947B0208958D
:10050000CF93C82F0E9479028C2F0E947D02CF9139
:10051000089580E00C9480020E944F1D0C9480028C
:100520000E944F1D9091A201891721F08093A20192
:100530000C9480020895CF93DF93CDB7DEB72B974D
:100540000FB6F894DEBF0FBECDBF4F8358876987C3
:100550007A878B8761110E94680C9E012F5F3F4F45
:1005600086E0F90111928A95E9F785E0FE01379658
:10057000D90101900D928A95E1F789819A814C8188
:100580005D81452B31F09F3F31F491E08F3F19F4AD
:1005900003C091E001C090E090FF09C049815A81F9
:1005A0006B817C818D819E810E94890B05C0C90170
:1005B0000E94FD018111F2CF2B960FB6F894DEBF99
:1005C0000FBECDBFDF91CF910895FC018081918155
:1005D0000E94B4080895CF93882309F4A9C0C82FB6
:1005E0008238C1F40E944F1D81FDA2C069E3809151
:1005F0000201909103010E94E91D0E948A0C2FEFD5
:1006000081EE94E0215080409040E1F700C000006E
:1006100069E319C0833801F50E944F1D80FD88C031
:1006200063E580910201909103010E94E91D0E94FF
:100630008A0C2FEF81EE94E0215080409040E1F74A
:1006400000C0000063E580910201909103010E94C7
:10065000EB1DCF910C948A0C8438C1F40E944F1D7D
:1006600082FD66C067E480910201909103010E94BF
:10067000E91D0E948A0C2FEF81EE94E0215080400A
:100680009040E1F700C0000067E4DDCF8CEF8C0FF5
:10069000813AF8F48C2F0E94441A811149C06C2FC2
:1006A00080910201909103010E94B31D882349F0BB
:1006B0006C2F80910201909103010E94EB1D0E941A
:1006C0008A0C6C2F80910201909103010E94E91D18
:1006D000C0CF80E28C0F883048F4C77081E001C041
:1006E000880FCA95EAF70E944B0CB3CFEBE5EC0FED
:1006F000E33040F4F0E0E25AFE4F808190E0CF9189
:100700000C947B1DE8E5EC0FE73150F4F0E0EE0FC0
:10071000FF1FE05DFE4F80819181CF910C94911D70
:10072000CD3E30F08C2F0E94A715CF910C947916F6
:10073000CF910895882309F464C0823879F40E9427
:100740004F1D81FF5EC069E380910201909103011A
:100750000E94E91D0E948A0C69E310C08338B1F43D
:100760000E944F1D80FF4DC063E580910201909172
:1007700003010E94E91D0E948A0C63E58091020139
:10078000909103010E94EB1D0C948A0C843879F43B
:100790000E944F1D82FF35C067E480910201909155
:1007A00003010E94E91D0E948A0C67E4E7CF9CEFD9
:1007B000980F913A10F4682FE1CF90E2980F98309B
:1007C00050F4877091E001C0990F8A95EAF7892F5C
:1007D0000E94510CD9CF9BE5980F933020F480E014
:1007E00090E00C947B1D98E5980F973120F480E001
:1007F00090E00C94911D8D3E20F00E9402160C9406
:10080000791608951F93CF93DF93182FEB010E9461
:10081000EB02209741F08FE99FE00197F1F700C0CC
:1008200000002197F6CF812FDF91CF911F910C947B
:100830009A03893319F060E070E002C060E570E06F
:100840000C940204882321F00E944B0C0C948A0C17
:100850000895882321F00E94510C0C948A0C08956D
:10086000CF92DF92EF92FF920F931F93CF93DF937C
:100870007C01D62FC72FFC011281058102950F70D4
:100880000E94410C8823B9F01123A9F08C2F807F9E
:10089000803421F080E28D0F883068F080919102E1
:1008A00082FD09C082E00E94EA0C0E94410C91E0A6
:1008B000D82ED92601C0D12CCC2EC2948FE0C822CC
:1008C0008C2D90E08C30910508F0CDC1FC01EA5AE6
:1008D000FF4F0C94FB258C2F807FCF70882311F065
:1008E000C295C07F112399F0CC2309F4A8C180E2FE
:1008F0008D0F883010F0D11104C08C2F0E944B0C4A
:1009000003C08C2F0E945B0C0E948A0C98C18D2F13
:100910000E949A03CC2309F4A6C180E28D0F88308F
:1009200038F1DD2329F18C2F0E94610C24C08C2F1B
:10093000807FCF70803211F0C295C07FDD2319F027
:10094000D130A1F13CC08091910282FF17C01123E8
:1009500049F0CC2329F08C2F0E944B0C0E948A0C6A
:1009600080E06EC180E00E949A03CC2309F47BC131
:100970008C2F0E94510C0E948A0C75C1112371F0BA
:10098000002341F0013031F40E946B0C8C2B0E944B
:10099000730C69C10E946B0C8C2B1CC0002319F0D6
:1009A000013009F460C10E94800C24C0112321F0A1
:1009B000023008F058C10DC0011155C11BC01123F0
:1009C00061F0002331F0F701858180FF38C18F701D
:1009D00085838C2F0E94220446C1002359F0D9330D
:1009E00009F03EC1FFEF07EE13E0F1500040104068
:1009F000E1F734C18C2F0E94290435C18C2F8695D4
:100A00008695837019F0813061F02DC1112321F09A
:100A10008D2F9C2F937002C080E090E00E947B1D80
:100A20002AC1112321F08D2F9C2F937002C080E0EA
:100A300090E00E94911D1FC18D2F112319F00E947B
:100A4000A71502C00E9402160E94791614C18C2FAD
:100A5000837009F047C011110AC12D2F22952695E8
:100A60002770220F220F6D2F6F70862F90E0A0E06D
:100A7000B0E0022E04C0880F991FAA1FBB1F0A9462
:100A8000D2F7D4FF10C04FE050E060E070E004C047
:100A9000440F551F661F771F2A95D2F74095509532
:100AA0006095709503C040E050E0BA01C695C695C8
:100AB000C3708A019B01082B192B2A2B3B2BC901E0
:100AC000B801C23049F058F4C13019F00E942F0724
:100AD000CEC00E941D07CBC00E944107C8C00E9423
:100AE0001B07C5C0112319F08C2F817001C086959A
:100AF000882309F4BCC02D2F229526952770220F3C
:100B0000220F6D2F6F70862F90E0A0E0B0E0022ED4
:100B100004C0880F991FAA1FBB1F0A94D2F7D4FFE5
:100B200010C04FE050E060E070E004C0440F551F7B
:100B3000661F771F2A95D2F740955095609570955E
:100B400003C040E050E0BA01C695C695C3708A0163
:100B50009B01082B192B2A2B3B2BC901B801C23052
:100B600049F058F4C13019F00E94F40780C00E9487
:100B7000E2077DC00E9406087AC00E94550777C030
:100B8000CF70112339F08C2F0E947B078D2F0E948C
:100B900022046DC08D2F0E9429048C2F0E949C0777
:100BA00066C0D23F19F128F4D03F41F0D13FB9F0EF
:100BB00042C0D33F11F1D43F71F03DC0112339F051
:100BC000011151C08C2F8F710E94C1074CC002309F
:100BD00008F049C0F7CF8091910282FF18C011231D
:100BE00039F08C2F8F710E947B073DC01123C9F310
:100BF0008C2F8F710E949C0736C0112329F08C2FF7
:100C00008F710E9466072FC00E9461072CC01123BC
:100C100049F0CF718C2F0E947B0763E08C2F0E94DC
:100C2000CF0C21C081E00E94EA0C0230E0F082E0AB
:100C30000E94EA0C18C0112331F0002391F28D2F8D
:100C40000E94EB0210C0002399F2D93349F41FEF40
:100C500027EE33E0115020403040E1F700C00000A3
:100C60008D2F0E949A0388EF8C0D843020F40E940F
:100C70004F1D0E948002DD20C9F00E943D0C80FDC6
:100C800015C0F70112820E94370C0E947B07C70132
:100C90000E9477060E94370CDF91CF911F910F9130
:100CA000FF90EF90DF90CF900C949C07DF91CF9155
:100CB0001F910F91FF90EF90DF90CF9008950F93C9
:100CC0001F93CF93DF93EC01688179818A810E9421
:100CD000BF088C010E9418080E940907B801CE01C4
:100CE0000E943004DF91CF911F910F910895CF930F
:100CF000DF93EC01988189812B813C81232B31F09A
:100D00008F3F31F481E09F3F19F403C081E001C0BF
:100D100080E080FD1DC0CE010E941E02811110C026
:100D20000E94410C8823A1F08A81882389F0809158
:100D3000910282FD0DC082E0DF91CF910C94EA0C0C
:100D4000CE010E945F06CE01DF91CF910C94FF018E
:100D5000DF91CF91089580E090E00E947B1D80E0BC
:100D600090E00E94911D0E94680C0E948A0C0E94D3
:100D7000AA170C94791680910201909103010E94A8
:100D8000ED1D0C94AB060E94580C0C94BB0692957A
:100D90009F70963079F010F4925001C09A509230C2
:100DA00068F4803F69F018F4883E40F409C0843F3D
:100DB00029F406C0883E20F0813F11F080E00895BC
:100DC00081E00895FC01808191810E94B4080E9415
:100DD000C7060895CF93DF9300D000D01F92CDB700
:100DE000DEB70F900F900F900F900F90DF91CF9183
:100DF0000895CF93DF9300D000D000D0CDB7DEB7F9
:100E000026960FB6F894DEBF0FBECDBFDF91CF910F
:100E10000895089508950C940A070C940B070E94F6
:100E20000D076093D5017093D6018093D7019093FD
:100E3000D8010C94AB060C940F070F931F930091ED
:100E4000D5011091D6012091D7013091D801602BA6
:100E5000712B822B932B1F910F910C940F070F93E3
:100E60001F930091D5011091D6012091D7013091A7
:100E7000D80160237123822393231F910F910C9437
:100E80000F070F931F930091D5011091D601209168
:100E9000D7013091D80160277127822793271F91AE
:100EA0000F910C940F070C940A070E94530760934C
:100EB000D1017093D2018093D3019093D4010C940B
:100EC000AB0660E070E0CB010C9455070F931F93C5
:100ED00041E050E060E070E08A019B0104C0000F37
:100EE000111F221F331F8A95D2F7C901B8011F9124
:100EF0000F910C9455070F931F9341E050E060E071
:100F000070E004C0440F551F661F771F8A95D2F703
:100F10008091D1019091D201A091D301B091D401DF
:100F20008A019B01082B192B2A2B3B2BC901B801E5
:100F30001F910F910C9455070F931F9341E050E0C0
:100F400060E070E004C0440F551F661F771F8A954C
:100F5000D2F740955095609570958091D101909110
:100F6000D201A091D301B091D4018A019B01082341
:100F700019232A233B23C901B8011F910F910C9417
:100F800055070F931F9341E050E060E070E004C00C
:100F9000440F551F661F771F8A95D2F78091D101A4
:100FA0009091D201A091D301B091D4018A019B010B
:100FB000082719272A273B27C901B8011F910F913C
:100FC0000C9455070F931F930091D1011091D201FA
:100FD0002091D3013091D401602B712B822B932B64
:100FE0001F910F910C9455070F931F930091D101FE
:100FF0001091D2012091D3013091D401602371234B
:10100000822393231F910F910C9455070F931F93E5
:101010000091D1011091D2012091D3013091D401DE
:1010200060277127822793271F910F910C945507F2
:101030000895292F220F920F990F890FE82FE69517
:10104000E695E695877051E001C0550F8A95EAF75D
:1010500085E0E89FF0011124EC55FE4F20E030E0E0
:1010600070E04081CB01022E02C0969587950A94CC
:10107000E2F78170819584278523842781932F5FF0
:101080003F4F2530310569F70895292F220F920F20
:10109000990F890F682F669566956695982F9770BA
:1010A00085E0689FB001112440E050E080E0FB0142
:1010B000E40FF51FEC55FE4F208130E0092E02C0F1
:1010C000369527950A94E2F721703327042E01C044
:1010D000220F0A94EAF7822B4F5F5F4F453051058C
:1010E00031F70895BF92CF92DF92EF92FF920F9364
:1010F0001F93CF93DF938C01C090D101D090D20188
:10110000E090D301F090D4018091D5019091D60167
:10111000A091D701B091D801C82AD92AEA2AFB2A7E
:10112000CFE1D0E0D701C6010C2E04C0B695A7953B
:10113000979587950A94D2F780FD04C0219790F780
:10114000B12C07C0BC2EB8018C2F0E94D80F01977C
:10115000A9F38B2DDF91CF911F910F91FF90EF900D
:10116000DF90CF90BF900895CF93DF93EC010E9462
:101170007208BE010E94D80FDF91CF9108951F938E
:10118000CF93DF93EB019091A301992321F0CB0141
:101190000E94B40813C0882349F0CB010E94720852
:1011A000182F682FCE010E94190804C0CB010E949D
:1011B0004508182FBE01812F0E94D80FDF91CF91D3
:1011C0001F9108951F93CF93DF93C091D90116E02B
:1011D0008091DA01C81799F0D0E01C9FF0011D9FA3
:1011E000F00D1124E552FE4F4081518162817381DF
:1011F000848195810E94F9062196C770E9CFDF911D
:10120000CF911F91089540910B0250910C02609173
:101210000D0270910E0280910F02909110020C94B9
:10122000F9062091D9019091DA0156E02917A9F029
:1012300030E0529FF001539FF00D1124E552FE4F14
:101240007181761306C07081781303C072817413A4
:1012500006C02F5F3F4F2770E9CF80E0089581E0FF
:101260000895EF92FF920F931F93CF93DF93809196
:10127000100282958F7009F065C080910D0288235D
:1012800009F460C08091D901F090DA0110910B024D
:1012900000910C0260910E0270910F0291E01F3FCD
:1012A00009F090E0C0910001D0910101292F96E052
:1012B000E92E8F1509F446C06115710521F00F3F25
:1012C00021F030E003C031E001C0322F90E030FD6A
:1012D00036C0E89EF001E99EF00D1124DF01A55211
:1012E000BE4F11963C911197301329C03C91311398
:1012F00026C012963C911297311121C013964D9140
:101300005C911497461B570B4C175D07C0F48091F6
:1013100010028F70806180931002E052FE4F808136
:101320008F70806180838BE092E00E947706DF916E
:10133000CF911F910F91FF90EF900C94E2080196CE
:101340008770B7CFDF91CF911F910F91FF90EF90F2
:1013500008958F929F92AF92BF92CF92DF92EF92B9
:10136000FF920F931F93CF93DF93CDB7DEB76197B3
:101370000FB6F894DEBF0FBECDBF8C0185E0F8013B
:10138000DE011D9601900D928A95E1F7D801129623
:10139000EC9090910B0220910C0240910E02509122
:1013A0000F024115510531F02F3F31F481E09F3F8D
:1013B00019F403C081E001C080E080FD7CC1F80128
:1013C000C080D180838094808BE0A82E82E0B82EEC
:1013D000F0900D02B401641B750B40910001509117
:1013E0000101FF2009F411C180911002382F307FD4
:1013F0006417750708F0CBC031118AC0D21214C02F
:10140000C91212C0FE2CE1100FC08F708061809352
:1014100010020E940309C5010E9477068091100204
:10142000D80115968C9361C18114910439F0BFEFF6
:10143000DB1206C081E0CB1203C003C081E001C013
:1014400080E080FD03C081E08E2502C080E090E056
:1014500080FF10C04E2D6D2D8C2D0E941109882308
:1014600049F08BE092E00E947706EBE0F2E086E044
:10147000DF019DC0892839F0BFEFDB1206C081E093
:10148000CB1203C003C081E001C080E080FD03C037
:1014900081E08E2502C080E090E0E82FE170BE2E52
:1014A00080FF2CC04E2D6D2D8C2D0E941109F82E21
:1014B000811124C0CD86DE868D859E850E94B4086C
:1014C000292F22952F70223018F0243090F405C077
:1014D0009F7059F0811109C008C19F7031F0D80187
:1014E00015969C91907F09F400C1805E883008F4C5
:1014F000FCC0C8010E947706FB2CF7C0FE2CEE2032
:1015000009F4F3C08091100281608093100254C0EE
:10151000D21206C0C91204C0E11002C0F80199C07D
:10152000C8010E94E206882361F1EE2051F120916A
:101530001002822F82958F7090E0029774F0809154
:101540000B0290910C0298878F8319869B868A865E
:101550002C87CE0107960E94770686E0F801ABE063
:10156000B2E001900D928A95E1F70E9431090E9444
:1015700003090AC0D21611F1C8010E94E2068111C6
:101580002CC0C8010E947706FF24F394AEC031112D
:10159000F1CF782D998A888AA6016E2D89890E94BB
:1015A000EA068BE092E00E94770686E0D5011D9264
:1015B0008A95E9F70E940309F12C97C0C912DCCF84
:1015C000E110DACFF8018583C8010E94770686E032
:1015D000D5011D928A95E9F788C0EE2091F22091FD
:1015E0001002822F82958F7090E002970CF4B5CF95
:1015F00080910B0290910C029A8389831B829D82B9
:101600008C822E83CE010196A6CF6417750708F051
:1016100044C0FE2CEE2009F4B4CFD21230C0C9125F
:101620002EC02091100220FD21C0822F82958F7044
:10163000482F50E041155105C9F0F80125834F307E
:10164000510541F08F5F982F9295907F822F8F7078
:10165000892B8583C8010E94770686E0F801ABE0FC
:10166000B2E001900D928A95E1F73DC086E0F80165
:10167000ABE0B2E001900D928A95E1F736C0C80167
:101680000E94E206811169CF8091100281608093EF
:101690001002C8010E94770628C0782D998A888A8E
:1016A000A6016E2D89890E94EA0686E0D5011D9269
:1016B0008A95E9F718C0EE2009F463CFC8010E94AB
:1016C000E206F82E882309F45CCF86E0F801ABE04F
:1016D000B2E001900D928A95E1F78BE092E00E94D2
:1016E000E5020E9431090E9403098F2D61960FB611
:1016F000F894DEBF0FBECDBFDF91CF911F910F9148
:10170000FF90EF90DF90CF90BF90AF909F908F9021
:1017100008951F93CF93DF93CDB7DEB72C970FB605
:10172000F894DEBF0FBECDBF4F83588769877A8795
:101730008B879C87CE0107960E94A9098823D1F048
:101740009F8188852A853B85232B31F08F3F31F49B
:1017500081E09F3F19F403C081E001C080E080FD7B
:1017600047C04F81588569857A858B859C850E9405
:10177000F9063EC086E0FE013796DE011196019023
:101780000D928A95E1F7FF81E8856A857B85611571
:10179000710531F0EF3F31F481E0FF3F19F403C0F0
:1017A00081E001C080E080FD23C02091DA0130E0BB
:1017B000C9010196877099274091D90150E084179B
:1017C0009507F1F1F983EA837D836C8396E0929F1C
:1017D000D001939FB00D1124A552BE4FFE0131964A
:1017E00001900D929A95E1F78093DA010E94E20848
:1017F00016E08091D9019091DA01891771F1189F53
:10180000C001112485529E4F0E94A909882329F105
:10181000E091D9011E9FF0011124E552FE4F408155
:10182000518162817381848195810E94F906809142
:10183000D90190E00196877099278093D901D9CF7B
:101840000E94C3061092DA011092D901EBE0F2E097
:1018500086E0DF011D928A95E9F72C960FB6F89481
:10186000DEBF0FBECDBFDF91CF911F910895809154
:10187000190285958595859508958091190287703F
:10188000089590911902977081E009F480E008951D
:1018900080912402089590912402892B8093240240
:1018A00008958095909124028923809324020895BD
:1018B00010922402089590912302892B8093230291
:1018C000089580959091230289238093230208959F
:1018D00010922302089580911A02089508950C949D
:1018E0006E0C0C946F0C9091910292FD08C0909137
:1018F0001A02981721F080931A020C94710C089523
:1019000080911A02882329F010921A0280E00C9428
:10191000710C0895CF93DF93E0910201F0910301E0
:10192000809124028083E0910201F0910301908173
:1019300080912302892B808380911A02882381F071
:10194000E0910201F09103019081892B80838091C5
:101950000201909103010E94A71D81110E94800C39
:10196000C0910201D091030148E050E061E172E0D2
:10197000CE010E941526892B69F088E0FE01A1E1C5
:10198000B2E001900D928A95E1F7CE01DF91CF91FF
:101990000C94621DDF91CF9108950C946E0C909180
:1019A000910292FD10C098E0899F90011124262B8E
:1019B000209319020E947B078091190285958595D5
:1019C00085950C94CD0C0C947B071092190280E045
:1019D0000C94CD0C209119028095822380931902DA
:1019E000982F977099F430E0482F082E000C550B73
:1019F0002417350759F09091910292FD07C0859503
:101A0000859585950E949C070C94E50C089590910E
:101A1000910292FB222720F9281769F080FB92F9A6
:101A20009093910280919002909191020E944F0DAB
:101A300082E00C94EA0C08958091910282FB882741
:101A400080F991E089270C94070D81E00C94070D33
:101A500080E00C94070D80E090E00E94332621E0A6
:101A6000893E9E4F09F020E0822F089582E090E0A9
:101A70000C942B2683E090E00C942B26CF9384E0EB
:101A800090E00E942B26C82F82E290E00E942B2635
:101A90002C2F30E0A901582BCA01CF910895CF9384
:101AA000C92F682F84E090E00E9439266C2F82E2D3
:101AB00090E0CF910C943926AB01BC018FE090E00F
:101AC0000C944B26AB01BC0183E190E00C944B26B7
:101AD00060E070E0CB010C94620D60E070E0CB013F
:101AE0000E945C0D0C94680D69EE7EEF80E090E042
:101AF0000E94572660E082E090E00E94392660E074
:101B000083E090E00E9439261092D5011092D60110
:101B10001092D7011092D80160E084E090E00E941A
:101B2000392660E082E290E00E94392660E085E09C
:101B300090E00E94392660E086E090E00E9439261D
:101B40006FEF87E090E00E94392640E050E0BA0154
:101B500088E090E00E944B2660E08DE090E00E94DB
:101B6000392640E050E0BA0188E190E00E944B261F
:101B700060E087E190E00E94392640E050E0BA0141
:101B80008CE190E00E944B2660E070E080E290E003
:101B90000E94572640E050E0BA0188E190E00E94A0
:101BA0004B260C946D0D0C94740D682F8EE090E014
:101BB0000C9439260E949B1E609335027093360266
:101BC000809337029093380260933102709332020F
:101BD0008093330290933402089585B7806885BF5F
:101BE00085B7806885BF08950C94E71208950C941A
:101BF000F60D0C94F60D0C94F90D0C94F60D0C9456
:101C0000FD0D0C94F60D0E94ED0D85EF90E10E9404
:101C1000451D0E94010E0C94FF0D0E94F70D0C94BF
:101C2000F60D0E94F8100C947F020E94861E0E94FE
:101C3000B4100E9401130E9438120E94110E0E94DB
:101C4000B8170E940B130C94FB0D8F929F92AF92CA
:101C5000BF92CF92DF92EF92FF920F931F93CF9399
:101C6000DF93CDB7DEB72A970FB6F894DEBF0FBE6D
:101C7000CDBF0E945C12982E81110E94DA0D85E280
:101C8000A82E82E0B82E00E010E0802E802F0E9467
:101C90001C11D82EF501C1905F01C826B1F40F5F69
:101CA0001F4F0C30110589F78FEF89838A831B82C0
:101CB0000E948F1E8160782F9D838C8349815A8179
:101CC0006B818D810E949B022FC08091390281FD22
:101CD0000E942211E12CFF24F3948C2D8F21F1F02E
:101CE0000E94F40D882399F0EE828F82DF2081E03C
:101CF00009F480E088870E948F1E8160782F9A8780
:101D000089874E815F8168858A850E949B02F801E0
:101D1000EB5DFD4F8081F826F08206C0E394FF0C56
:101D2000F6E0EF12DACFBBCF81E0911001C080E086
:101D30002A960FB6F894DEBF0FBECDBFDF91CF91CC
:101D40001F910F91FF90EF90DF90CF90BF90AF90D9
:101D50009F908F9008950E94250E0E94E7120E9486
:101D600097160C949002CF93DF930E94DD0FEC0145
:101D7000811521E5920708F045C0811530E59307EC
:101D800008F094C0883E910528F5803E910508F042
:101D9000F8C0883A910570F4853A910508F07CC046
:101DA0008130910509F475C008F4E8C0049708F083
:101DB000E8C0E4C08F3B910508F0E0C0C85AD0E00D
:101DC000CC0FDD1FCF59DE4F0990D881C02DCE0139
:101DD0009464D8C0811540E2940758F4811551E00D
:101DE000950708F0CEC08D3E910508F4C7C09065F8
:101DF000C9C0C11580E4D80708F4C0C0DF70CE01A7
:101E0000906AC0C0811525E59207A8F4811534E5D4
:101E1000930708F095C0811543E5940708F07BC04F
:101E2000811552E5950708F061C0D82FCC27CE0167
:101E3000816F906AA7C0C11589E5D807A0F4C115C4
:101E400028E5D20708F082C0C11536E5D30708F0AF
:101E500095C08C2F0E9471108F7190E0D82FCC27E5
:101E6000CE0190628FC0C1154AE5D40708F474C052
:101E7000CE0190568115904208F080C08D2F8F7151
:101E80000E947110DD27D0628F71AE01582BCA01FC
:101E900079C081E090E076C0C55AD0E0C157DE4FEE
:101EA0008881C82FD0E0CE0190646CC074E0969514
:101EB00087957A95E1F7282F23703C2F337081E0C6
:101EC00090E002C0880F991F3A95E2F79C68AC0138
:101ED000522B9A019C2F9F709695969550E2959F54
:101EE000E0011124C9018C2B9D2B4CC083709927D4
:101EF00021E030E002C0220F331F8A95E2F79C2FC9
:101F00009695969580E2989FE0011124C22BD32BE1
:101F1000CE019C6837C08370992721E030E002C071
:101F2000220F331F8A95E2F79C2F9695969540E2F3
:101F3000949FE0011124C22BD32BCE019A6822C0BA
:101F4000D82FCC27CE01846F906A1CC0DC2FCC2701
:101F5000CE01806F906A16C08C2F8F700E94711016
:101F600094E0D695C7959A95E1F7CF70D0E0DC2F35
:101F7000CC27D0699E01282BC90104C080E090E0E5
:101F800001C0CE01DF91CF91089528E4829FC00166
:101F90001124FC0126E0729FE00DF11D1124E60FD3
:101FA000F11DEE0FFF1FE852FF4F859194910895A8
:101FB0000E94C50F0E94B30E08958238910569F101
:101FC000B0F48133910509F46DC048F4893291056C
:101FD00009F463C08A32910509F469C00895853314
:101FE000910509F455C089339105B9F00895833EF0
:101FF000910569F138F4803E9105B1F0823E91057A
:1020000009F10895863E9105A9F1873E9105B9F140
:10201000843E910509F064C023C02091900220FD08
:102020004FC021FD4DC008958091900280FD44C0B5
:102030008091910280FF44C08091900284FD42C053
:1020400083EE4DC08091900282FF38C0F5CF809121
:10205000900282FD33C08091910280FD31C0ECCFAF
:102060008091910281FF32C08091900284FD2AC04C
:1020700087EE35C08091900283FF26C0F5CF809116
:10208000900283FD21C08091910281FD1FC0ECCFA1
:102090008091900285FD1CC01DC08091900285FD3D
:1020A00019C016C08091900286FD16C017C080919D
:1020B000900286FD13C010C089E311C082EE0FC0EC
:1020C00080EE0DC080E00BC086EE09C084EE07C034
:1020D00089E205C085E303C08AE201C081E390E0A4
:1020E00008959091900292FF0DC0282F28712830FA
:1020F00019F4877F846006C0282F2471243011F4DE
:102100008B7F886093FF0DC0282F2871283119F428
:10211000877E846106C0282F2471243111F48B7EC0
:1021200088612091910220FF0DC0382F387138301E
:1021300019F4877F816006C0382F3171313011F476
:102140008E7F886021FF0DC0282F2871283119F457
:10215000877E816106C0282F2171213111F48E7E86
:10216000886194FD877E089510928C0210928D02F2
:1021700010928E0210928F020895CF92DF92EF920A
:10218000FF926B017C010E94E71281110EC00E9438
:102190009B1EC61AD70AE80AF90AC0928C02D0928E
:1021A0008D02E0928E02F0928F02FF90EF90DF900E
:1021B000CF9008950F931F930E94E712882321F078
:1021C0001F910F910C949B1E0E949B1E00918C02EC
:1021D00010918D0220918E0230918F02600F711F3D
:1021E000821F931F1F910F91089580E00895089515
:1021F0000E942B0D811102C00E94D30D0E94360D4A
:10220000809339020E943E0D909391028093900238
:102210000E94F7100E943A0D682F70E080E090E075
:102220000E941B076091D1017091D2018091D3016E
:102230009091D4010C945307E82FF0E0E156FD4F44
:1022400080810895089580EA8A95F1F7089500C085
:1022500008950C94231108950C942B110C942C11B7
:102260000C942B110C9430110C942B11FF920F93A2
:102270001F93CF93DF9300D000D000D0CDB7DEB74F
:102280000E94E7126091AB028823E9F186E0F82E04
:102290008E010F5F1F4FF8018F2D11928A95E9F77C
:1022A000862F90E0B80181569D4F0E941913882314
:1022B00089F08091920290E046E050E0B8018156AA
:1022C0009D4F0E94152621E020933A02892B61F44C
:1022D00010E016C080913A028823D1F3F8011192E0
:1022E000FA94E9F710923A02A0919202B0E0A15656
:1022F000BD4F86E0F80101900D928A95E1F711E05B
:102300000E940C020DC070E061567D4F80919202D8
:1023100090E081569D4F0E94A3130E94341110E05B
:10232000812F26960FB6F894DEBF0FBECDBFDF918A
:10233000CF911F910F91FF900895F894E82FE295A7
:10234000EF70F0E031A1282F2F7081E090E001C004
:10235000880F2A95EAF7982F9095932391A392A13D
:10236000892B82A3789408950F931F93CF93DF93C3
:10237000C8E9D1E089918F3F11F00E949D1181E061
:10238000CE39D807B9F7C2E9D1E008E911E089915F
:102390008F3F11F00E949D110C171D07C1F7DF91AF
:1023A000CF911F910F910895CF92DF92EF92FF92FC
:1023B0000F931F93CF93DF938C01C62FD0E0CE01F4
:1023C00088569E4F7C01FC0190819F3F09F447C0D5
:1023D000D62EF894E92FE295EF70F0E081A19F707E
:1023E00021E030E001C0220F9A95EAF7822B81A309
:1023F00082A12095282322A378940E942711E2E944
:10240000F1E048E951E031E0C12C21912F3F89F002
:10241000A22FA295AF70B0E090968C9190E02F70B3
:1024200002C0959587952A95E2F780FD02C0832F1B
:1024300001C080E0C82A330F4E175F0731F7F7015C
:1024400080818F3F11F00E949D1161E0C11001C099
:1024500060E08D2D0E942911C00FD11FC882DF912D
:10246000CF911F910F91FF90EF90DF90CF90089543
:102470008091040180910401811102C096E001C0A5
:1024800090E09093AB0286E0891B809392020E94B9
:10249000B4118CE0EFE9F2E0DF01982F1D929A95DC
:1024A000E9F7E3E9F2E0DF011D928A95E9F786E0BA
:1024B0000E94B0120C940A02EF92FF920F931F93A6
:1024C000CF93DF93CDB7DEB72C970FB6F894DEBF6E
:1024D0000FBECDBF8E010F5F1F4F8CE0F801119230
:1024E0008A95E9F7F12C6F2DC8010E94D411F3945D
:1024F000F6E0FF12F8CF4CE050E0B80183E992E03B
:102500000E9415267C0121E0892B09F420E0E114CA
:10251000F10441F08CE0F801A3E9B2E001900D92E2
:102520008A95E1F76091AB0270E061567D4F46E01D
:1025300083E992E00E94B112EF2819F40E9436114B
:1025400002C081E090E02C960FB6F894DEBF0FBE7B
:10255000CDBFDF91CF911F910F91FF90EF90089524
:102560000895FF920F931F93CF93DF938C01F62E64
:10257000D72FC42F222349F081E080933D020E948F
:102580008F1E90933C0280933B0280913D028823F2
:10259000C1F080913B0290913C020E94A71E0597DA
:1025A00080F0EF2DFD2FD8014C2F50E0CD01801B86
:1025B000910B841795071CF48D918193F7CF10929E
:1025C0003D02DF91CF911F910F91FF90089580916F
:1025D000400281110DC00E94DA25811102C082E003
:1025E00001C081E080934002823011F40E94D52521
:1025F00081E090914002913009F080E008950C94C0
:10260000E7120E94FF12809304010E94E7128111D9
:102610000C94511308950E94E712811102C00C948A
:102620005313089581E0909141029A3008F080E0C0
:1026300008950F931F93CF93DF93EC018B0180914B
:1026400041028A3038F4B801CE010E94A1138111F1
:102650001DC00AC080913E0290913F020E94A71EB9
:10266000843F914080F715C0809141028F3F19F05F
:102670008F5F80934102809141028A3060F00E9416
:102680008F1E90933F0280933E0203C0109241023E
:1026900002C080E001C081E0DF91CF911F910F91D6
:1026A00008950C94DE1B0C94E11BDF92EF92FF92D5
:1026B0000F931F93CF93DF937901C82F880FDD0B02
:1026C00041155105A9F0FE0193E0EE0FFF1F9A9509
:1026D000E1F7EB5FFE4F818192818E5B9D4F208100
:1026E00030E04217530708F49A01A9010E942226FC
:1026F000CE010E94CA1CD82E8823D1F001151105E5
:10270000B9F083E0CC0FDD1F8A95E1F7FE01EB5FA6
:10271000FE4F438150E00417150708F4A801CB5F72
:10272000DE4F6C817D816E5B7D4FC7010E9422264A
:102730008D2DDF91CF911F910F91FF90EF90DF9042
:1027400008950C94C0140C94DC140F931F93CF9332
:10275000DF9300D000D0CDB7DEB760915B027091FF
:102760005C0280915D0290915E020E94B61E64360A
:1027700071058105910528F10E94DA10DC01CB0179
:102780000296A11DB11D89839A83AB83BC8300E0AF
:1027900010E020E030E044E050E0BE016F5F7F4F8A
:1027A00082E00E945513182F882361F00E949B1E1F
:1027B00060935B0270935C0280935D0290935E0273
:1027C00001C011E0812F0F900F900F900F90DF91BB
:1027D000CF911F910F910895AF92BF92CF92DF9248
:1027E000EF92FF920F931F93CF93DF937C015B01D6
:1027F0006A010E941213811103C001E010E002C0BF
:102800000AE010E0C1E0D0E0F894B501C701F6019C
:1028100009957894811115C021960C171D0794F025
:10282000CC9F9001CD9F300D300D112480E090E0C1
:1028300045E34A95F1F70000019682179307C1F727
:10284000E3CF81E0DF91CF911F910F91FF90EF9047
:10285000DF90CF90BF90AF900895AF92BF92CF928C
:10286000DF92EF92FF920F931F93CF93DF93CDB739
:10287000DEB727970FB6F894DEBF0FBECDBF7B0142
:10288000C0909E01D0909F0101E010E09E01295F61
:102890003F4F40E050E060E070E080E00E94551360
:1028A000182F882309F43EC056018FEFA81AB80AE2
:1028B00060915702709158028091590290915A028A
:1028C0000E94B61E643671058105910518F106E077
:1028D00010E09E012F5F3F4F40E050E060E070E06D
:1028E00081E00E945513182F66E070E0C5010E9438
:1028F000B91791E02F81281390E0192339F10E9434
:102900009B1E6093570270935802809359029093D4
:102910005A0211C066E070E0C5010E94B9179F819C
:102920008913D5CF86E0F6013196DE01119601902C
:102930000D928A95E1F7112349F086E0FE01319668
:10294000A1E5B2E001900D928A95E1F786E0E1E51C
:10295000F2E0D70101900D928A95E1F7812F279639
:102960000FB6F894DEBF0FBECDBFDF91CF911F91A0
:102970000F91FF90EF90DF90CF90BF90AF900895B0
:102980000F931F93CF93DF93EC018B014DE254E142
:102990000E94EC13882351F045EA53E1B801CE01BF
:1029A000DF91CF911F910F910C94EC1380E0DF9198
:1029B000CF911F910F9108950F931F93CF93DF93A2
:1029C000F894C0919E01D0919F01CE01019626E01E
:1029D000FB01DC0101900D922A95E1F766E070E0C1
:1029E0000E94B91788837894F8946F8178858985D7
:1029F0009A8500914D0210914E0220914F02309124
:102A00005002601771078207930751F060934D02DF
:102A100070934E0280934F02909350020E94BD101B
:102A20007894DF91CF911F910F9108950E949B2080
:102A30000E94150E0C94A7200E94AB200E94AB0EA2
:102A40000C94C5200E942D1E0E9482200E94030E1D
:102A50000E9416150E941C150E940D0EFBCF80913E
:102A6000670280FF06C06091210170E0660F771F4A
:102A700026C081FF04C06091210184E005C082FF6F
:102A800007C06091210188E0689FB001112417C040
:102A9000909166029923D1F060912001961788F7F2
:102AA0002091210188E0289F90011124929FA0018C
:102AB000939F500D112470E0CA010E94E7256038F1
:102AC000710540F46115710519F406C068E070E005
:102AD000862F08958FE7089581E008958091670219
:102AE00080FF08C060911E0170E07595679575952F
:102AF000679521C081FF06C060911E0170E0759549
:102B0000679519C082FF04C060911E0170E010C07B
:102B100090916502992399F060911D019617A0F795
:102B200080911E01899FC001112470E00E94E72559
:102B30006038710540F46115710519F406C061E053
:102B400070E0862F08958FE7089581E008958D3E07
:102B500021F40E942F15819504C08E3E29F40E9415
:102B60002F1580936B0208958F3E21F40E942F153C
:102B7000819504C0803F29F40E942F1580936A023A
:102B80000895893F19F40E946E1505C08A3F31F4FB
:102B90000E946E15819580936C0208958B3F21F4FD
:102BA0000E946E15819504C08C3F29F40E946E1519
:102BB00080936D0208959FE0980F983078F421E09B
:102BC00030E0A90102C0440F551F9A95E2F7CA01EF
:102BD00090916902892B8093690208958D3F21F4B9
:102BE0008091670281600BC08E3F21F48091670263
:102BF000826005C08F3F29F48091670284608093D2
:102C0000670208958D3E39F490916B0297FF35C0AD
:102C100010926B0259C08E3E29F490916B021916E6
:102C2000BCF32BC090916A028F3E29F497FF25C018
:102C300010926A0249C0803F19F41916CCF31DC0E6
:102C400090916C02893F29F41916BCF410926C0221
:102C50003BC08A3F19F497FF10C0F8CF8B3F39F47F
:102C600090916D0297FF09C010926D022DC08C3FAC
:102C700021F490916D021916BCF39FE0980F9830E3
:102C800080F421E030E0A90102C0440F551F9A955D
:102C9000E2F7CA01809590916902892380936902C5
:102CA00013C08D3F21F4809167028E7F0BC08E3F51
:102CB00021F4809167028D7F05C08F3F29F48091B8
:102CC00067028B7F8093670280916A02811106C040
:102CD00080916B02811102C01092660280916C0299
:102CE000811106C080916D02811102C010926502AF
:102CF00008950E948F1E20916A02211104C0209124
:102D00006B02222321F0909364028093630220914E
:102D10006C02211104C020916D02222321F09093B6
:102D200062028093610288E692E00C946D1DEF923E
:102D3000FF920F931F93CF93DF9300D000D000D06A
:102D4000CDB7DEB786E0E8E6F2E0DE01119601904D
:102D50000D928A95E1F7E0906A02F0906B02009183
:102D60006C0210916D0210926A0210926B02109226
:102D70006C0210926D02E11003C0FF2009F45DC0E7
:102D800080916302909164020E94A71EAC01909111
:102D90006602992339F02091220130E0241735078B
:102DA00058F04BC0209160028AE0289F90011124C6
:102DB0002417350718F041C09F3F19F09F5F90938B
:102DC0006602EE2061F00E942F151E1414F09FEF92
:102DD00001C091E0989F902D112490936A02FF20EA
:102DE00061F00E942F151F1414F09FEF01C091E0B5
:102DF000989F902D112490936B0230916A02332397
:102E0000E1F020916B022223C1F045EB3403C001B5
:102E10001124992319F090936A0203C081E08093F2
:102E20006A0235EB2303C0011124992319F0909312
:102E30006B0203C081E080936B02011103C0112378
:102E400009F45DC080916102909162020E94A71E08
:102E5000AC0190916502992339F020911F0130E077
:102E60002417350758F04BC020915F028AE0289F55
:102E7000900111242417350718F041C09F3F19F025
:102E80009F5F90936502002361F00E946E151016FB
:102E900014F09FEF01C091E0989F902D1124909322
:102EA0006C02112361F00E946E15111614F09FEF51
:102EB00001C091E0989F902D112490936D02309164
:102EC0006C023323E1F020916D022223C1F045EB27
:102ED0003403C0011124992319F090936C0203C0AC
:102EE00081E080936C0235EB2303C0011124992308
:102EF00019F090936D0203C081E080936D02809180
:102F00006A0281110BC080916B02811107C0809110
:102F10006C02811103C080916D0281110E947916AB
:102F2000EB82FC820D831E8386E0FE013196A8E6CB
:102F3000B2E001900D928A95E1F726960FB6F894CB
:102F4000DEBF0FBECDBFDF91CF911F910F91FF90DC
:102F5000EF900895E8E6F2E086E0DF011D928A95A1
:102F6000E9F71092660210926502109267020895C6
:102F70000895FC01680F791F8FEF91E3E617F707BB
:102F800071F02191822728E030E087FF03C0880F8D
:102F9000892701C0880F21503109B9F7EFCF089573
:102FA000CF93DF93EC01FB018281882309F43CC1BC
:102FB000C430FDE5DF0760F4CB3F9CE5D90788F41A
:102FC0009E0122503C452431310508F02EC109C034
:102FD000C236EDE5DE0729F0C63AFDE5DF0709F068
:102FE00024C10E943E0D9093910280939002C131C2
:102FF0008CE5D80709F4C6C008F042C0C930ECE53A
:10300000DE0709F49BC000F5C5308CE5D80709F44C
:1030100085C078F4C330ECE5DE0709F478C008F029
:103020007AC0C230DC4509F0F5C080919002816021
:10303000EFC0C7309CE5D90709F478C008F07AC022
:10304000809190028061E4C0CD30FCE5DF0709F497
:1030500087C058F4CB309CE5D90709F479C008F053
:103060007BC08091900288606FC0CF30FCE5DF07A5
:1030700009F480C008F082C080919002877FC8C0A8
:10308000CE3F9CE5D90709F471C000F5C531FCE5D8
:10309000DF0709F485C068F4C3319CE5D90709F45A
:1030A00075C008F095C00E94C306809190028F778A
:1030B000AFC0CC3FFCE5DF07A9F108F054C0CB3F1F
:1030C000DC4509F0A7C08091910240C0C230EDE517
:1030D000DE0709F489C058F4C1158DE5D80709F455
:1030E0005AC008F069C08091910282602FC0C23638
:1030F000EDE5DE0709F47CC0C63AFDE5DF0709F41B
:1031000081C0C330DD4509F085C080E06EC080918C
:10311000900282607DC08091900216C080919002E2
:10312000886076C08091910282604FC08091900249
:1031300080626EC08091900280646AC00E94C30663
:1031400080919002806864C0846062C081603DC0EC
:10315000809190028E7F5CC0809190028D7F58C0DC
:103160008091900216C08091910218C080919102C6
:103170008D7F2BC0809190028F7E4AC080919002FB
:103180008F7D46C0809190028F7B42C080919002DB
:10319000877F8B7F3DC0809191028D7F8E7F15C090
:1031A0008091900282FB222720F991E0922790FBE8
:1031B00082F990FB83F92CC080919102982F909511
:1031C00091708E7F892B90FB81F98093910222C0B0
:1031D0000E94C3068091900287FB222720F991E08C
:1031E000922790FB87F914C081E00E94D50D12C090
:1031F0008091900284FB222720F991E0922790FB96
:1032000084F906C080919002982F909590FB80F9E8
:103210008093900280919002909191020E944F0DB4
:103220000E94C30680E001C081E0DF91CF91089544
:10323000893279F1E0F4843161F1A0F4873009F04A
:1032400075C01092600294E1909322018093210155
:103250008EE18093200188E080931E0188E28093B4
:103260001D0164C092EE980F9A30F0F05FC0803577
:1032700009F444C028F48F3409F058C08AE03FC0F4
:10328000813529F0823509F051C081E038C08FEFD7
:1032900036C080917002882379F1109270021092EA
:1032A0006F0210926E0242C08D5180937002833083
:1032B00099F038F4813069F08230D9F482E291E0FB
:1032C0000DC0853099F078F0863099F48DE191E069
:1032D00005C080E692E002C081E291E090936F0227
:1032E00080936E0223C080E291E0F8CF8EE191E0FE
:1032F000F5CF109270021AC080E0089586EFE09139
:103300006E02F0916F02309789F02081082E000C38
:10331000990B820F911D8F3F910519F014F08FEFDB
:1033200004C097FF02C0108201C0808381E008952D
:103330000F931F9341E050E060E070E08A019B0131
:1033400004C0000F111F221F331F8A95D2F7C90135
:10335000B8010E941B071F910F910C94C3068B317B
:1033600009F468C058F58B3009F486C078F48630CB
:1033700009F445C020F4853009F44BC07FC0873084
:1033800009F44AC0883009F477C078C0803109F464
:1033900064C068F48E3009F071C08091390282FBFC
:1033A000222720F991E0922790FB82F94CC08631C8
:1033B00009F462C0893109F45FC060C08A32E1F06B
:1033C00060F4873209F455C028F48E3108F456C0F1
:1033D0008D5150C08932E9F051C0833450F48A33A2
:1033E00008F045C0853309F444C0883309F444C06B
:1033F00045C08334F1F142C00E94D30D3DC080919D
:103400003902817F8E7F8093390281E0809371023F
:1034100008950E940F0230C080913902982F909534
:10342000917090FB80F980933902911125C0897FBA
:10343000877F10C08091390281FB222720F991E01B
:10344000922790FB81F9809339029923A9F080910A
:1034500039028160809339020FC08091390283FB69
:10346000222720F991E0922790FB83F9ECCF895332
:1034700001C080E00E94981981E0089580E00895DD
:1034800080E008950C94401ACF93C82F8091710268
:10349000813069F038F08230C1F58C2F0E94181904
:1034A00081E039C00E94480C823289F504C00E9434
:1034B000480C823261F48C2F0E94421A811104C0A0
:1034C0008C2F0E94AF191FC081E090E01CC08C2F90
:1034D0000E94401A811116C0C43189F058F4CB30D3
:1034E00089F0C031B1F482E08093710288E30E94D8
:1034F000181908C0C93219F0C83321F00AC0109257
:10350000710207C081E0817006C01092710280E0F4
:1035100002C080E0F8CFCF910895CF93DF9386313A
:103520009C4541F5EB010E94480C982F8A8120911F
:10353000020130910301882379F09A7A81E009F43D
:1035400080E080937202911102C069E201C065E3DC
:10355000C9010E94E91D0AC080917202811102C056
:1035600069E201C065E3C9010E94EB1D0E948A0C5B
:1035700080E001C081E0DF91CF9108950F931F9308
:10358000CF93DF93C42FD22FFC0182818823C9F00F
:10359000409375020E948F1E909374028093730271
:1035A00080E28C0F883008F057C0C77081E001C0FE
:1035B000880FCA95EAF7DF91CF911F910F910C9474
:1035C000220480917502481330C08091730290915B
:1035D00074020E94A71E883C910538F510E21D0F69
:1035E000CD17B9F080E28C0F883040F4C77081E0CD
:1035F00001C0880FCA95EAF70E942904183028F5FF
:1036000081E09D2F977001C0880F9A95EAF70E947C
:103610002204802F0E9419041830F0F4D77081E042
:1036200001C0880FDA95EAF70AC080E28C0F883073
:1036300098F4C77081E001C0880FCA95EAF7DF915E
:10364000CF911F910F910C942904802FDF91CF917E
:103650001F910F910C941904DF91CF911F910F913D
:1036600008950F939C01CB01243F4CE5340731F1C1
:1036700088F4293DFCE53F07D9F02A3D4CE53407A5
:1036800079F1283D3C45A9F506E221EE41EE68EDD1
:103690007CE52BC0263FFCE53F07E1F0A8F0273F83
:1036A0003C4539F507E225EE46EE67EF7CE51DC0A7
:1036B00007E225EE45EE69ED7CE517C006E221EE56
:1036C00040EE64EF7CE511C007E225EE44EE65EFC5
:1036D0007CE50BC006E221EE42EE66EF7CE505C01C
:1036E00008E221E045EE6AED7CE50E94BE1A80E02A
:1036F00008C0FC018281882319F01092750201C074
:1037000081E00F9108958EE1489B02C08150E1F75E
:10371000489BFECF0895589880E28A95F1F7589A11
:103720000895FC012AE02A95F1F728E090E080E076
:1037300031E040E14A95F1F7880F489B02C0816073
:10374000932700C0000040E14A95F1F7215089F726
:1037500020E12A95F1F729B100C0000030E13A9547
:10376000F1F7217092272081920F90830895EF92B4
:10377000FF920F931F93CF93DF931F92CDB7DEB7C6
:1037800019828C017C01E60EF11C0E151F0551F00B
:103790000E94831BCE0101960E94911BF801819328
:1037A0008F01F3CF81E09981911180E00F90DF913B
:1037B000CF911F910F91FF90EF900895509A589AD2
:1037C00008955098589AE89AE9E6F0E080818C7F55
:1037D00080830895615091E001C0990F6A95EAF7DE
:1037E00020E031E0992361F0492F482319F0589ADD
:1037F000232701C0589840E24A95F1F79695F2CFF9
:10380000222311F0589A01C0589880E28A95F1F766
:1038100058980895FF920F931F93CF93DF93EC0175
:103820008C01060F111DC017D10741F0F9900E94BD
:103830008B1B68E08F2D0E94EA1BF5CFDF91CF91A3
:103840001F910F91FF9008951F920F920FB60F9244
:1038500011240F931F932F933F934F935F936F9375
:103860007F938F939F93AF93BF93EF93FF93CF93E8
:10387000DF931F92CDB7DEB719820E94831BCE0162
:1038800001960E94911B082F069506950695902F8C
:1038900096959570202F2570920F292F237096955D
:1038A0009695920F877089135FC0898181115CC0E2
:1038B000043008F059C080E18A95F1F7589A509A7F
:1038C00082E08A95F1F700C0589888E0089F80014F
:1038D0001124D801AB5FBE4F1696ED91FC9117975E
:1038E0003097A9F060919E0170919F0114962D91DF
:1038F0003C911597260F371F11968D919C91129729
:10390000680F791F13964C9113978C910995F801C4
:10391000EB5FFE4F6381662351F080919E01909191
:103920009F0124813581820F931F0E940A1C0E94EF
:103930008B1B80E18A95F1F758985098589A80E14E
:103940008A95F1F7F801EB5FFE4F6081662351F035
:1039500080919E0190919F0121813281820F931F5E
:103960000E94B71B0E94831B0F90DF91CF91FF91A4
:10397000EF91BF91AF919F918F917F916F915F91E7
:103980004F913F912F911F910F910F900FBE0F906C
:103990001F9018950F931F93CF93DF938430910559
:1039A0000CF06DC0EC01F894509A589885E08A9517
:1039B000F1F700009C2F969595702C2F2570920F93
:1039C000892F83709695969523E0CC0FDD1F2A955D
:1039D000E1F7980F8E01092B0E948B1B84E08A95DA
:1039E000F1F700C068E0802F0E94EA1B80E18A9511
:1039F000F1F75098589A489902C000C0FCCF87E070
:103A000090E0489B08C0019721F4509A589A789406
:103A100036C000C0F6CFFE01EB5FFE4F6381662328
:103A200081F080919E0190919F0124813581820FC8
:103A3000931F0E94B71B811104C0509A589A789422
:103A40001FC00E94831B80E28A95F1F75898509A14
:103A500080E18A95F1F7CB5FDE4F6881662351F0F4
:103A600080919E0190919F0129813A81820F931F3D
:103A70000E940A1C0E948B1B789481E001C080E0A8
:103A8000DF91CF911F910F9108959093A1018093A1
:103A9000A001089590937C0280937B0208950E9478
:103AA000E712811103C0809176020895E0917B02B4
:103AB000F0917C02309721F00190F081E02D099483
:103AC00080E00895E0917B02F0917C02309721F034
:103AD0000280F381E02D09940895E0917B02F0913A
:103AE0007C02309739F022E0DC012C930480F581D0
:103AF000E02D099408952091790230917A022817D7
:103B0000390771F090937A0280937902E0917B02F9
:103B1000F0917C02309721F00680F781E02D099426
:103B2000089520917702309178022817390771F0B3
:103B30009093780280937702E0917B02F0917C026F
:103B4000309721F00084F185E02D09940895FC015F
:103B5000329697E080E0915029F021912223D9F309
:103B60008F5FF9CF0895662349F0FC0132960896DD
:103B70002191621729F0E817F907D1F780E008953D
:103B800081E008959C01FC0132969FEF80E0419115
:103B9000461789F09F3F19F4411101C0982F8F5F9C
:103BA0008630A9F79F3F39F0F901E90FF11D97FD24
:103BB000FA956283089508959C012A5F3F4FFC01A6
:103BC0004281461301C01282019682179307B9F70A
:103BD00008950C94C21D0C94DC1D029626E0FC0195
:103BE00011922A95E9F7089508950C94F41D83E045
:103BF00080937D020C94F51D811102C081E001C00B
:103C000082E080937D020C94F51D0C94FC1D81E0F4
:103C100080937D020C94F51D0C94071E08950C945E
:103C20000E1E0C940F1E0C940E1E0C940E1E0C9463
:103C30000E1ECF930E94151E0E945C120E94131E3E
:103C4000C0E08C2F0E941C11811104C0CF5FCC30CA
:103C5000C1F701C081E0CF91089508951F920F929E
:103C60000FB60F9211248F939F93AF93BF938091C0
:103C70007E02811113C08091AC029091AD02A0919F
:103C8000AE02B091AF024196A11DB11D8093AC026E
:103C90009093AD02A093AE02B093AF02BF91AF91EB
:103CA0009F918F910F900FBE0F901F90189580914C
:103CB000B402843031F10E94700210927E0220E43E
:103CC00088E190E00FB6F894A895809360000FBE4D
:103CD0002093600083B7817F846083BF83B7816056
:103CE00083BF7894889583B78E7F83BF0FB6F8948F
:103CF000A8958091600088618093600010926000B8
:103D00000FBE08950E94C3060C94740282E084BD25
:103D100093E095BD9AEF97BD80936E0008952FB7FD
:103D2000F8948091AC029091AD02A091AE02B09156
:103D3000AF022FBF08952FB7F8946091AC02709135
:103D4000AD028091AE029091AF022FBF08959C0109
:103D50004FB7F8948091AC029091AD02A091AE0261
:103D6000B091AF024FBF821B930B0895CF92DF92A9
:103D7000EF92FF922FB7F894C090AC02D090AD02B2
:103D8000E090AE02F090AF022FBFA7019601261B74
:103D9000370B480B590BCA01B901FF90EF90DF9028
:103DA000CF90089578941F920F920FB60F9211241E
:103DB0008F939F93AF93BF938091AC029091AD028C
:103DC000A091AE02B091AF020196A11DB11D8093EA
:103DD000AC029093AD02A093AE02B093AF02BF913C
:103DE000AF919F918F910F900FBE0F901F901895DC
:103DF00087E797E790930108809300089AE088E1AD
:103E00000FB6F894A895809360000FBE9093600061
:103E1000FFCF80918A020895089522E02093E9005F
:103E20002FEF3091E800215035FD06C035ED3A9571
:103E3000F1F700002111F5CF2091E80025FF0BC01C
:103E400040E050E066E070E00E9437218091E80099
:103E50008E778093E8000895CF93DF9321E020933D
:103E6000E9002FEF3091E800215035FD06C035ED17
:103E70003A95F1F700002111F5CF2091E80025FFD8
:103E800014C0EC0140E050E068E070E00E9437218F
:103E90008091E8008E778093E80088E0FE01A2E838
:103EA000B2E001900D928A95E1F7DF91CF910895EC
:103EB00080937F0270938102609380028091B402AC
:103EC000843001F582E08093E9008FEF9091E80063
:103ED000815095FD06C095ED9A95F1F7000081118E
:103EE000F5CF8091E80085FF0DC040E050E063E031
:103EF00070E08FE792E00E9437218091E8008E7792
:103F00008093E8000895BC0184E00C94581FBC0124
:103F100083E00C94581F8091B302811109C00E9464
:103F2000C8220E9425238091E20084608093E200F1
:103F300008951092B30208950C940C1E6091B00283
:103F400081E0611101C080E00C94F71D9091B402F2
:103F500081E0943009F080E06091B0020C94FC1D87
:103F600042E061EC81E00E94412242E261EC82E0A9
:103F70000E9441229091B40281E0943009F080E0E7
:103F80006091B0020C94051E8091B602833009F452
:103F900061C030F4813071F0823009F49AC0089524
:103FA0008A3009F486C08B3009F46CC0893009F07E
:103FB000A8C020C08091B502813A09F0A2C08091CA
:103FC000E800877F8093E8008091B9029091BA025F
:103FD000892B21F468E082E892E003C060E080E091
:103FE00090E070E00E9482218091E8008B778093BE
:103FF000E80008958091B502813209F082C0809175
:10400000B9029091BA02029708F07BC08091E80053
:10401000877F8093E8008091E80082FD05C0809151
:10402000B4028111F8CF6DC02091F3008091F200AD
:1040300090E0922B029731F48091F100813011F0E1
:10404000863021F48091F10080938A028091E8000B
:104050008B7753C08091B502813A09F052C08091AC
:10406000B9029091BA02892B09F04BC08091E80007
:10407000877F8093E8008091E80080FFFCCF8091EB
:104080002F0136C08091B5028132D9F58091B902F5
:104090009091BA02892BA9F58091E800877F8093DF
:1040A000E8000E9476228091B70280932F010C9441
:1040B000C3068091B502813221F58091E800877FA7
:1040C0008093E8000E9476228091B80280938B0250
:1040D00008958091B502813AA1F48091E800877F2C
:1040E0008093E8008091E80080FFFCCF80918B02F4
:1040F0008093F1008091E8008E778093E8000C9423
:104100007622089584B7877F84BF0FB6F894A89568
:1041100080916000886180936000109260000FBE03
:1041200090E080E80FB6F89480936100909361006E
:104130000FBE0C94071E0E94C8220E942523E2EEA7
:10414000F0E080818460808378940C94BA2583E2C7
:1041500091E00C944A1D8091B4028530A9F48091BD
:10416000B402853079F40E94571E8091B2028823F0
:10417000B1F30E94191E882391F30E9421210E940D
:10418000C306EDCF0C94821E089508950C94C820A8
:10419000292F332723303105C9F060F42130310550
:1041A00081F02230310509F044C08BE390E02AE22F
:1041B00032E043C021323105E1F02232310549F1CC
:1041C00038C082E190E025E632E037C0992781309F
:1041D000910549F028F0029761F5E8EFF1E005C09C
:1041E000E6E2F2E002C0E0E1F2E0849190E09F01BB
:1041F00024C06115710541F061307105D1F489E089
:1042000090E025E532E019C089E090E02CE332E04F
:1042100014C06115710541F06130710551F48BE7EF
:1042200090E027E732E009C080E490E022EF32E03E
:1042300004C080E090E020E030E0FA013183208388
:10424000089580E189BD82E189BD09B400FEFDCFFA
:104250008091D8008F7D8093D8008091E0008260AB
:104260008093E0008091E00081FDFCCF0895CF9223
:10427000DF92EF92FF920F931F93CF93DF93EC01A6
:104280008B017A010E949522811133C0E114F1045F
:1042900039F0F70180819181081B190BC80FD91FD4
:1042A000C12CD12C0115110519F18091E80085FD73
:1042B00016C08091E8008E778093E800E114F10445
:1042C00049F0F70180819181C80ED91ED182C08248
:1042D00085E00FC00E949522882321F30AC08991AE
:1042E0008093F10001501109FFEFCF1ADF0ADACFF6
:1042F00080E0DF91CF911F910F91FF90EF90DF90C1
:10430000CF9008952091BB023091BC022617370749
:1043100048F06115710539F42091E8002E7720935B
:10432000E80001C0B901FC0120E06115710579F1D7
:104330008091B4028823F1F18530F1F18091E80099
:1043400083FD3CC08091E80082FD2EC08091E80092
:1043500080FFEBCF2091F3008091F20090E0922B50
:104360006115710551F08830910538F42191209341
:10437000F100615071090196F3CF21E0089709F02F
:1043800020E08091E8008E778093E800CECF211165
:10439000CFCF0AC08091B402882361F0853061F0EC
:1043A0008091E80083FD0AC08091E80082FFF2CF8F
:1043B00080E0089582E0089583E0089581E0089503
:1043C0002091BB023091BC022617370748F06115D7
:1043D000710539F42091E8002E772093E80001C0A0
:1043E000B901FC0120E06115710591F18091B402E1
:1043F000882309F440C0853009F43FC08091E8006B
:1044000083FD3DC08091E80082FD2FC08091E800CF
:1044100080FFE9CF2091F3008091F20090E0922B91
:104420006115710559F08830910540F4249120936D
:10443000F1003196615071090196F2CF21E00897A1
:1044400009F020E08091E8008E778093E800CBCFE0
:104450002111CCCF0AC08091B402882361F085304D
:1044600061F08091E80083FD0AC08091E80082FF3E
:10447000F2CF80E0089582E0089583E0089581E01E
:104480000895982F973068F59093E900981739F0C0
:104490007091EC002091ED005091F00003C0242FAA
:1044A000762F50E021FD02C09F5FECCF3091EB00F2
:1044B0003E7F3093EB003091ED003D7F3093ED0077
:1044C0003091EB0031603093EB007093EC0020935F
:1044D000ED005093F0002091EE0027FDE5CF80E045
:1044E00008958F708093E90081E008958091B5026E
:1044F00087FF11C08091E80082FD05C08091B40261
:104500008111F8CF11C08091E8008B770BC08091AA
:10451000B402882349F08091E80080FFF8CF8091B1
:10452000E8008E778093E80008952091E4003091B0
:10453000E50095E64091EC00842F817040FF23C098
:104540008091E80080FD1DC08091B402882399F01D
:10455000853099F08091EB0085FD11C04091E40019
:104560005091E5002417350729F3915011F09A0175
:10457000E1CF84E0089582E0089583E0089581E02A
:10458000089580E008954091E80042FFDDCF08954E
:104590000E9436230E943E23E0EEF0E0808181609D
:1045A0008083E8EDF0E080818F77808319BCA7EDF0
:1045B000B0E08C918E7F8C9380818F7E808310926F
:1045C000B30208950F931F93CF93DF930E94362376
:1045D0000E943E23C8EDD0E088818F778883888150
:1045E0008068888388818F7D888319BC1092B4028B
:1045F0001092B0021092B2021092B10200EE10E0DE
:10460000F80180818B7F808388818160888342E08C
:1046100060E080E00E944122E1EEF0E080818E7F48
:104620008083E2EEF0E08081816080838081886019
:104630008083F80180818E7F808388818061888378
:10464000DF91CF911F910F910895E8EDF0E0808107
:104650008F7E8083E7EDF0E080818160808384E05D
:1046600082BF81E08093B3020C94E222E8EDF0E097
:1046700080818E7F80831092E20008951092DA008C
:104680001092E10008951F920F920FB60F9211241D
:104690002F933F934F935F936F937F938F939F934A
:1046A000AF93BF93EF93FF938091E10082FF0BC024
:1046B0008091E20082FF07C08091E1008B7F8093B0
:1046C000E1000E94B9258091DA0080FF1FC080912F
:1046D000D80080FF1BC08091DA008E7F8093DA00C3
:1046E0008091D90080FF0DC080E189BD82E189BD44
:1046F00009B400FEFDCF81E08093B4020E948B1FBD
:1047000005C019BC1092B4020E94991F8091E1006B
:1047100080FF19C08091E20080FF15C08091E20007
:104720008E7F8093E2008091E20080618093E200BE
:104730008091D80080628093D80019BC85E0809376
:10474000B4020E949E1F8091E10084FF30C08091DE
:10475000E20084FF2CC080E189BD82E189BD09B4FB
:1047600000FEFDCF8091D8008F7D8093D80080918E
:10477000E1008F7E8093E1008091E2008F7E809344
:10478000E2008091E20081608093E2008091B002BB
:10479000882311F084E007C08091E30087FD02C008
:1047A00081E001C083E08093B4020E94A61F809143
:1047B000E10083FF29C08091E20083FF25C0809142
:1047C000E100877F8093E10082E08093B402109241
:1047D000B0028091E1008E7F8093E1008091E20041
:1047E0008E7F8093E2008091E20080618093E200FE
:1047F00042E060E080E00E9441228091F000886009
:104800008093F0000E949C1FFF91EF91BF91AF91A8
:104810009F918F917F916F915F914F913F912F91D8
:104820000F900FBE0F901F9018951F920F920FB60A
:104830000F9211242F933F934F935F936F937F9326
:104840008F939F93AF93BF93CF93DF93EF93FF9398
:10485000C091E900CF708091EC00D82FD17080FD1D
:10486000D0E81092E9008091F000877F8093F000FB
:1048700078940E9459241092E9008091F000886099
:104880008093F000CD2BCF70C093E900FF91EF91A2
:10489000DF91CF91BF91AF919F918F917F916F9158
:1048A0005F914F913F912F910F900FBE0F901F90EE
:1048B00018951F93CF93DF93CDB7DEB7AA970FB6A6
:1048C000F894DEBF0FBECDBFE5EBF2E08091F100C2
:1048D000819322E0ED3BF207C9F70E94C41F80914B
:1048E000E80083FF2EC18091B5029091B602492F56
:1048F00050E04A30510508F024C1FA01EE59FF4F4B
:104900000C94FB25803821F0823809F01AC108C0C8
:104910008091B1029091B202992389F082600FC018
:104920008091B9028F70873008F00BC18093E90045
:104930008091EB0085FB882780F91092E900909127
:10494000E800977F9093E8008093F1001092F100C7
:10495000D1C0282F2D7F09F0F4C0882319F08230B0
:1049600061F0EFC08091B702813009F0EAC0933066
:1049700009F080E08093B2022EC08091B7028111CD
:104980002AC08091B9028F702FEF280F263008F0CF
:10499000D8C08093E9002091EB0020FF1CC0933029
:1049A00021F48091EB00806214C09091EB00906143
:1049B0009093EB0021E030E0A90102C0440F551FA5
:1049C0008A95E2F74093EA001092EA008091EB00AA
:1049D00088608093EB001092E9008091E800877F67
:1049E0008093E8000E947622ACC08111AAC0109189
:1049F000B7021F778091E3008078812B8093E300DA
:104A00008091E800877F8093E8000E947622809161
:104A1000E80080FFFCCF8091E30080688093E30092
:104A2000111102C082E001C083E08093B40289C00A
:104A30008058823008F085C08091B7029091B8020A
:104A40008C3D53E0950779F583E08A838AE2898378
:104A50004FB7F894DE01139620E03EE051E2E32FD9
:104A6000F0E050935700E49120FF03C0E295EF700F
:104A70003F5FEF708E2F90E0EA3010F0C79601C0D4
:104A8000C0968D939D932F5F243149F74FBF80913E
:104A9000E800877F8093E8006AE270E0CE0101962B
:104AA0000E94822116C06091B9027091BA02AE01D3
:104AB0004F5F5F4F0E94C620BC01892B09F441C0A3
:104AC0009091E800977F9093E80089819A810E94F5
:104AD000E0218091E8008B778093E80032C0803835
:104AE00081F58091E800877F8093E8008091B00293
:104AF0008093F1008091E8008E7772CF811121C000
:104B00008091B7029091B80299270297D4F48091CE
:104B1000E800877F8093E8008091B7028093B0021D
:104B20000E9476228091B002811106C08091E3003C
:104B300087FD02C081E001C084E08093B4020E943E
:104B4000B01F8091E80083FF0AC08091E800877F52
:104B50008093E8008091EB0080628093EB00AA963E
:104B60000FB6F894DEBF0FBECDBFDF91CF911F917E
:104B700008950895CF938091B4028823A1F0C09145
:104B8000E900CF709091EC00892F817090FD80E852
:104B9000C82B1092E9008091E80083FD0E945924FF
:104BA000CF70C093E900CF9108950E94C82210925F
:104BB000B4020895E8EDF0E08081806180838AE1AD
:104BC0008A95F1F700C08091D9008170089597FB14
:104BD000072E16F4009407D077FD09D00E94012615
:104BE00007FC05D03EF4909581959F4F08957095F0
:104BF00061957F4F0895EE0FFF1F0590F491E02D12
:104C00000994AA1BBB1B51E107C0AA1FBB1FA61713
:104C1000B70710F0A61BB70B881F991F5A95A9F765
:104C200080959095BC01CD010895FB01DC0104C085
:104C30008D910190801921F441505040C8F7881B94
:104C4000990B0895FB01DC0102C001900D924150C7
:104C50005040D8F70895F999FECF92BD81BDF89ADA
:104C6000992780B50895A8E1B0E042E050E00C94A7
:104C70005F26262FF999FECF92BD81BDF89A019744
:104C800000B4021639F01FBA20BD0FB6F894FA9A94
:104C9000F99A0FBE08950396272F0E943A260E9484
:104CA0003926252F0E943A26242F0C943A26019665
:104CB000272F0E943A260C943926DC01CB01FC01F7
:104CC000F999FECF06C0F2BDE1BDF89A319600B465
:0E4CD0000D9241505040B8F70895F894FFCF70
:104CDE00C8001B02010000000100000000000000DF
:104CEE000601000000040700000000000028085024
:104CFE001E0714091F2C1F0D1F871F831F0C1F015A
:104D0E00E200E900EA00B500B600B700CD0083016D
:104D1E00CC008A0192019401210223022402250271
:104D2E00260227022A02B300B4006F0070008182AF
:104D3E0083E200E900EA00B500B600B700CD0083BB
:104D4E0001CC008A01920194012102230224022542
:104D5E0002260227022A02B300B4006F00700081FF
:104D6E008283946697C63435F6F731333236420273
:00000001FF
